:030000000243D4E4
:0C43D40078FFE4F6D8FD75815A02441B06
:10288D000A53746172743A20004950436F6E6E653D
:10289D0063745245510A00444843502D4F4B0A0072
:1028AD004950436F6E6E65637400C0E4E0EFF2E56E
:1028BD00F020D1E8EDEAEEEC4950284343290A0017
:1028CD00C2E5F0F1E8FF20495020ECEEE4F3EBFF18
:1028DD003A20322E3420EEF22032302E31312E328B
:1028ED003030350A00C4E0F2E020F1EEE7E4E0ED2F
:1028FD00E8FF3A20005365702032362032303036F2
:10290D0000200031313A32323A3136000A000A5095
:10291D00524F473A20202020202020202020202008
:10292D00202020202020202020202020202020209A
:10293D00202020202020202020202020202020208A
:10294D00202020202020202020202020202020207A
:10295D002020202020202020200A0044756D705852
:10296D0020202020203030203031203032203033D4
:10297D00203034203035203036203037203038208C
:10298D003039203041203042203043203044203037
:10299D00452030460A003A200044756D70442020D1
:1029AD002020203030203031203032203033203084
:1029BD003420303520303620303720303820303933
:1029CD0020304120304220304320304420304520FB
:1029DD0030460A00457272206B657900526420659D
:1029ED006570726F6D0A005264204D454D0A0044AA
:1029FD00656275674950204F4E0A004465627567E0
:102A0D004950204F46460A00446562756755736507
:102A1D0072204F6E0A0044656275675573657220AA
:102A2D004F46460A0044656275674D7367204F6EC9
:102A3D000A0044656275674D7367204F46460A006C
:102A4D00436F6E666967206C6F636B210A00577266
:102A5D0020656570726F6D0A002053617665206583
:102A6D006570726F6D210A00457272204D414321D0
:102A7D00004C6F61643E3E0057616974526573741A
:102A8D0061727421004E4F4950004C494E4B434FDB
:102A9D004E5452005452415353004652004E4F4C27
:102AAD00494E4B00494E490000FF2A92FF2A97FFDD
:0E2ABD002AA1FF2AA7FF2AAAFF2AB1FF2AB5E5
:064DCE0001560001540033
:104D6700C2AFC28E758900438910758BFF758DB7E9
:074D7700D2ABD28ED2AF22B5
:03001B0002433E5F
:10433E00C0E0C083C082C0D0C2AFC28E758BFF7585
:10434E008DB720060675A61E75A6E10554D202E5A8
:10435E0056600205560559E559540F7053D20DE5B6
:10436E0059543F7014D20090660CE0600C04F0E0DB
:10437E00D394B44004C2AF80FE906607E06002049E
:10438E00F0E555D3940140021555906104E06002AA
:10439E0014F090660DE0D394014003E014F0300564
:1043AE00020557E558D394644004D206800205589E
:1043BE00E553D3940140021553D28ED2AFD0D0D054
:0643CE0082D083D0E03232
:104BC100E4FFFEFD74DA2DF582E43462F583E02F13
:104BD100FFE43EFE0DBD10ECE4FD742F2DF582E4E3
:104BE1003461F583E0FC2FFFE43EFEEC60040DBD73
:024BF10080E85A
:014BF300229F
:100BAB00C291C290C20A7D027C007F07124D148F46
:100BBB0024E524646060097D017F60124CAFD20A8A
:100BCB00E4FDFC7F0B124D148F24E52430E6097DE8
:100BDB0004E4FF124CD3D20A7D017C007F07124D37
:100BEB00148F24E5247008FD7FFF124CAFD20A301E
:100BFB000A03126000C2AFC288D2A8C2AA12477FF2
:100C0B00C291D290D2AF124BC1123112D291C2907B
:100C1B0090660812259800000000E47F207E4EFDB0
:100C2B00FC906608E0F8A3E0F9A3E0FAA3E0FBC3AD
:100C3B001225655027906608E0FCA3E0FDA3E0FEBB
:100C4B00A3E0FFE4FAF9F8EF2401FFEA3EFEE93DE9
:100C5B00FDE83CFC90660812258C80BED291D290A8
:100C6B00124460C206C291D290124A8AD291C290AB
:100C7B009062D8E0C3940350037403F0D20CD20BF0
:100C8B00D20AD293200A077E287F8D123F53E4901D
:100C9B0064F8F0124D67C2AF755501A3F0C207C2DD
:100CAB0008D2AF75A70775A61E75A6E1124D31D2F6
:100CBB0091D29090660812259800000000E47F20E6
:100CCB007E4EFDFC906608E0F8A3E0F9A3E0FAA3E2
:100CDB00E0FBC31225655027906608E0FCA3E0FDFE
:100CEB00A3E0FEA3E0FFE4FAF9F8EF2401FFEA3EEC
:100CFB00FEE93DFDE83CFC90660812258C80BEC2E7
:100D0B0091C290200A19AF247E007D03124038E473
:100D1B00FF1241EE7E627FF8E4FB7D0112411690DB
:100D2B00660CE060037401F0E4906104F0A3745569
:100D3B00F0A37481F0E4F557E4F558906104E0708A
:100D4B0003122CF590660DE0B40111908000741025
:100D5B00F0E490660DF0D20AD20BD20CE557D39487
:100D6B0003402D908002E4F0908001F0908000F021
:100D7B00E557D3940540037401F0E557D3940A402B
:100D8B000FE4F557C2039064F9F0755501124A8AC6
:100D9B009080A0E070077FCB7E0312467F9080B8D7
:100DAB00E0700312429C9080D0E07014300E1190D2
:100DBB00660374FFF09062CCE0FEA3E0FF1247F4F1
:100DCB00908000E07013300710123E479062B4EF32
:100DDB00F0D394004003121A60908002E0700690EA
:100DEB008000E06005D205020D43C205E4F5579083
:100DFB006104E06003020D43300915123932906231
:100E0B00B4EFF0D394004008300105E0FF124DA37E
:100E1B002008030210221236499062B4EFF07003DF
:100E2B00020D4390660CE060037401F09062F8E0F1
:100E3B0054BF247F7003020EF6147003020ED724E6
:100E4B00026003020FCD200A077E287F96123F53C4
:100E5B009062D0E0FF70069062D4E060559066031C
:100E6B00E0FEB50722A3E0FF9062D1E0B507189032
:100E7B006605E0FF9062D2E0B5070C906606E0FFD6
:100E8B009062D3E06F602B9062D4E06E7035906609
:100E9B0004E0FF9062D5E0B50729906605E0FF906E
:100EAB0062D6E0B5071D906606E0FF9062D7E0B50D
:100EBB000711C2039064F97403F0120021755501F8
:100ECB0002102290660374FFF00210229065FBE083
:100EDB00FF9062FAE06F60030210229065FBE00462
:100EEB00F0E4F5559064F8F0021022300303021081
:100EFB00229062F9E0D3940A5003020FA0A3E0649E
:100F0B00026003020FA09062C1E0FF906303E06FE9
:100F1B006003020D439062C2E0FF906304E06F60D8
:100F2B0003020D439062C3E0FF906305E06F600323
:100F3B00020D439062C4E0FF906306E06F60030212
:100F4B000D439062C5E0FF906307E06F6003020DF5
:100F5B00439062C6E0FF906308E06F6003020D43AD
:100F6B007E287FA4123F539062FB63A2019062B96B
:100F7B0063A2017F121233CE90630D63A2019066C0
:100F8B000363A2017F041233CE9064F97406F075EB
:100F9B005502020D4374C744627003020D43124D98
:100FAB00D5D203E4F5559064F8F090660704F0E4AD
:100FBB009065FAF0A3F0200A5E7E287FAD123F53B6
:100FCB0080553003529062F8E020E74B9062FAE0D4
:100FDB00FF9065FAE0FE6F600D906602E07007EE21
:100FEB00146F703380139065FAE004F09062B4E0F4
:100FFB00FFD394044003124B8D9060007482F0A3D6
:10100B007401F09062FAE0906002F07E607F007DE8
:10101B0003124700020D432003030210DE9080D021
:10102B00E0700B9062CCE0FEA3E0FF1247F4E555B5
:10103B007066906607E0D3943C4037906602E07090
:10104B00311200069066077401F0E49063F8F0A388
:10105B007412F09065FBE09063FAF0A374FDF090CE
:10106B00610763A2019063FC63A2017F121233CE6E
:10107B008006124BF4EF60207E637FF89063F9E0FB
:10108B002404FD124700906602E06003020D4390BA
:10109B0062D8E0F555020D43124DB2EF601590602A
:1010AB00007483F0E4A3F07E607F007D02124700A2
:1010BB00020D43E55564016003020D439064F8E0B3
:1010CB0004F0E0C3940540B0C203E4A3F012002186
:1010DB00020D43E55564016003020D439064F9E092
:1010EB001470030211821470030211AE1470030208
:1010FB00125614700302130C24FE6069240660035D
:10110B00020D43E4F557F52474B02524F582E4343D
:10111B0061F583E0FF74B92524F582E43462F5832D
:10112B00EFF00524E524B43FDF200E219062D0635D
:10113B00A20190660363A2017F041233CE9064F97F
:10114B007401F09064F8F0755503020D439064F947
:10115B007404F09064F87401F07555149066037480
:10116B00FFF0020D43E4F557124A8A9064F97401BB
:10117B00F0755503020D43906603E0600B9062CC53
:10118B00E0FEA3E0FF1247F47555029064F9740278
:10119B00F09062C7E07003020D439064F97403F0A2
:1011AB00020D43906603E070030212479063F874DC
:1011BB0080F09063FA7402F0E4A3F0A304F0906261
:1011CB00C163A2019063FD63A2017F0A1233CE902B
:1011DB0064077430F0A3747BF0E4F524742F25249A
:1011EB00F582E43461F583E0FF601174092524F581
:1011FB0082E43464F583EFF0052480E07409252440
:10120B00F582E43464F583747DF0740A2524F58249
:10121B00E43464F583E4F0E52424119063F9F07C65
:10122B00667D039062CCE0FAA3E0FB7F021245FBE4
:10123B007E637FF8E5242413FD1247009064F97454
:10124B0004F09062D8E0F555020D43906603E07010
:10125B00030212FD9063F87480F09063FA7401F04E
:10126B00E4A3F0A304F0A37430F0A3747BF0E4F5D3
:10127B0024742F2524F582E43461F583E0FF60119B
:10128B0074FF2524F582E43463F583EFF0052480A5
:10129B00E074FF2524F582E43463F583747DF074E8
:1012AB00002524F582E43464F583E4F0E524240777
:1012BB009063F9F07C667D039062CCE0FAA3E0FBCF
:1012CB007F021245FB7E637FF8E5242409FD12475C
:1012DB0000906602E0601B124DD5D203E4F55590E9
:1012EB0064F8F090660704F0E49065FAF0A3F0025E
:1012FB000D439064F97404F09062D8E0F555020D3B
:10130B0043906603E0FF6009F4600690800274105E
:10131B00F0200E2B7555029064F8E06401FFF0A3EA
:10132B007401F0EF60059062D080039062D463A2E9
:10133B000190660363A2017F041233CE020D437545
:0D134B00551490660374FFF0020D4380FE00
:011358002272
:101A60009062F9E0B444047F0180027F009062F844
:101A7000E0B447047E0180027E00EE5F604A90621F
:101A8000C1E09062FAF09062C2E09062FBF0906276
:101A9000C3E09062FCF09062C4E09062FDF090625E
:101AA000C5E09062FEF09062C6E09062FFF0906246
:101AB000F97452F09062AE63A2019080A863A20113
:101AC0007F061233CE021F6E9062B4E0C3940850BA
:101AD00003021F779062C1E0FF9062FAE06F60033B
:101AE000021F779062C2E0FF9062FBE06F6003022A
:101AF0001F779062C3E0FF9062FCE06F6003021FFB
:101B0000779062C4E0FF9062FDE06F6003021F7790
:101B10009062C5E0FF9062FEE06F6003021F779065
:101B200062C6E0FF9062FFE06F6003021F7790667D
:101B30000CE060037401F090660D7464F09062F93B
:101B40007452F09062F8E0644D703C7E287FB712CA
:101B50003F537E287FCD123F53124DC67E287FF221
:101B6000123F537E297F02123F537E297F0E123F80
:101B7000537E297F10123F537E297F19123F537ED7
:101B8000297F1B123F53229062F8E0644C70527E12
:101B9000297F68123F53906300E0F525A3E0F52606
:101BA000E4F5277D03AF26AE251240387E297FA3BA
:101BB000123F53AE25AF26E4FB7D101241167E295D
:101BC0007F19123F5374102526F526E43525F52597
:101BD0000527E527C3941040CA7E297F19123F5379
:101BE000229062F8E0646C705CF5297E297FA61271
:101BF0003F53E4F528AF297E007D031240387E294B
:101C00007FA3123F53E4F527A829E6FF7402252796
:101C1000F582E43463F583EFF005290527E527B461
:101C200010E67E637F02E4FB7D101241167E297F61
:101C300019123F530528E528C3940840B87E297F30
:101C400019123F53229062F8E0644B7046F52774F6
:101C5000EA2527F582E43462F583E0FF601674001C
:101C60002527F582E43463F583E0B507100527E501
:101C700027B408DB9061047432F0021F6E9062F8A2
:101C80007421F0300A03021F6E7E297FE1123F5358
:101C9000021F6E9062F8E06452704E200A077E299F
:101CA0007FE9123F53906301E09062B4F0E4F527BE
:101CB0009062B4E0FDE527C39D5022906300E025CB
:101CC0002724AFF582E43461F583E0FF7402252711
:101CD000F582E43463F583EFF0052780D37E627FDD
:101CE000F8ED240AFD124575229062F8E06449700F
:101CF00045200A077E297FF4123F53906300E0F5E8
:101D000025A3E0F526E4F527852682852583E0FFD7
:101D100074022527F582E43463F583EFF00526E5A8
:101D200026700205250527E527B480DC7E627FF852
:101D30007D8A124575229062F8E064446003021DBA
:101D4000C7906300E0FF64447003021F6EEFB4317C
:101D50000CC20A7E297FFC123F53021F6E90630063
:101D6000E0B4300CD20A7E2A7F08123F53021F6E65
:101D7000906300E0B4320CD20B7E2A7F15123F53E1
:101D8000021F6E906300E0B4330CC20B7E2A7F23E7
:101D9000123F53021F6E906300E0B4340CD20C7EED
:101DA0002A7F32123F53021F6E906300E0B4350C5D
:101DB000C20C7E2A7F3F123F53021F6E906300E0E9
:101DC000FF12001E021F6E906104E07013200A07CC
:101DD0007E2A7F4D123F539062F87421F0021F6EED
:101DE0009061047432F09062F8E0FFB45104C2AF25
:101DF00080FEEF64577045200A077E2A7F5B123F02
:101E000053906301E09062B4F0E4F5279062B4E08F
:101E1000FFE527C39F4003021F6E74022527F5824A
:101E2000E43463F583E0FF906300E0252724AFF5F9
:101E300082E43461F583EFF0052780D09062F8E00A
:101E400064536003021EE9200A077E2A7F66123F60
:101E5000539062C1E0FF9061B8E06F703C9062C245
:101E6000E0FF9061B9E06F70309062C3E0FF906175
:101E7000BAE0B507249062C4E0FF9061BBE0B5070B
:101E8000189062C5E0FF9061BCE0B5070C9062C697
:101E9000E0FF9061BDE06F60169062F87421F03051
:101EA0000A03021F6E7E2A7F75123F53021F6EE4E3
:101EB000F527E4F55874AF2527F582E43461F583FE
:101EC000E0FDAF27124D4D0527E527C394FE40E204
:101ED000C2AFE4907FF0F0A3F0907FFD74AAF0A36E
:101EE00074FFF0A37455F080FE9062F8E0644F70C8
:101EF0004B906300E0F525A3E0F526E52645257027
:101F00000A200A077E2A7F7E123F53200A077F2A73
:101F10007E00123F53E4F52774022527F582E4344E
:101F200063F583E0852682852583F00526E5267006
:101F30000205250527E527B480DE80329062F8E0AF
:101F4000B4452B200A077E2A7F85123F53906300F9
:101F5000E0FFA3E0907FF0CFF0A3EFF0C2AF907F5F
:101F6000FD74AAF0A374FFF0A37455F080FE7E62A6
:071F70007FF87D08124575A2
:011F77002247
:104B5500AE07EEC39430400BEED394395005EE24E6
:104B6500D0FF22EEC39461400BEED394665005EE60
:104B750024A9FF22EEC39441400BEED39446500581
:084B8500EE24C9FF22AF062255
:10311200C201E490660CF0D20EC204906602F090F6
:1031220062C163A2019065FC63A2017F061233CEE5
:10313200E4F525E52575F003A424B6F582E4342AE6
:10314200F583E493FB740193FA740293F912242D2C
:1031520070030232F2E4F526F527FD742F2DF58275
:10316200E43461F583E0FF70030232EDE52575F08A
:1031720003A424B6F582E4342AF583E493FB7401B4
:1031820093FA740293F9852682758300122446FE0F
:10319200EFB5060875270105260232E9E527700317
:1031A2000232E9EE60030232E4E52524FE602214D5
:1031B20070030232D41470030232D8147003023244
:1031C200E0240460030232ED90660C7401F00232D6
:1031D200EDD201742F2DF582E43461F583E0FF64B2
:1031E2002D70030232ED124B55EFC454F0FC7430D3
:1031F2002DF582E43461F583E0FF124B55EF2C90FC
:1032020065FCF074312DF582E43461F583E0FF1240
:103212004B55EFC454F0FC74322DF582E43461F561
:1032220083E0FF124B55EF2C9065FDF074332DF5C2
:1032320082E43461F583E0FF124B55EFC454F0FC95
:1032420074342DF582E43461F583E0FF124B55EFBF
:103252002C9065FEF074352DF582E43461F583E03F
:10326200FF124B55EFC454F0FC74362DF582E43452
:1032720061F583E0FF124B55EF2C9065FFF0743738
:103282002DF582E43461F583E0FF124B55EFC4540F
:10329200F0FC74382DF582E43461F583E0FF124BC3
:1032A20055EF2C906600F074392DF582E43461F507
:1032B20083E0FF124B55EFC454F0FC743A2DF582B3
:1032C200E43461F583E0FF124B55EF2C906601F078
:1032D2008019D20480159066027401F0800DC20E2E
:1032E2008009E4F527F5260D02315D052502313509
:0132F20022B9
:030003000249238C
:0D492300C0E0C083C082C0D075D000C007C6
:10493000C2A8908008E0FFEF54F06035EF30E40843
:10494000D2079080087410F0EF30E508D20990800B
:10495000087420F0EF30E608D2089080087440F028
:10496000EF30E7069080087480F0908008E0FF80C8
:09497000C690800874FFF0D2A883
:0B497900D007D0D0D082D083D0E03235
:104A8A009080007480F09062B963A201F583F58288
:104A9A0063A2017F081233CE9062C163A2019080A3
:104AAA008863A2017F0A1233CE9062CBE0FF908026
:104ABA00B1F09080E1EFF09080957455F0A3F090FA
:0C4ACA0080007401F09080097470F022EC
:04467F00AD07AC06D1
:10468300908009E04410F09080A0E0706F9080A1CA
:104693007482F09080A874FFF0A3F0A3F0A3F0AFAE
:1046A30004AE079080AEEEF0AE05A3EEF0AE079039
:1046B30080ACEEF0AE05A3EEF09080007402F090B3
:1046C3006BB812259800000000906BB8E090804012
:1046D300F0906BB9E0908041F0906BBAE09080422B
:1046E300F0906BBBE0908043F0A3E4F0A3F0A3F061
:0C46F300A3F0908018F0A3F0A3F0A3F057
:0146FF002298
:0447F400AD07AC065B
:1047F800908009E04440F09080D0E070559080D1DE
:104808007482F0AF049080DEEFF0AF05A3EFF09074
:1048180080027402F0906BBC122598000000009092
:104828006BBCE0908058F0906BBDE0908059F090A0
:104838006BBEE090805AF0906BBFE090805BF0A375
:10484800E4F0A3F0A3F0A3F0908030F0A3F0A3F07D
:02485800A3F0CB
:01485A00223B
:10429C00908009E04420F09080B8E0600302433D38
:1042AC009080B97482F07F039080C6EFF07FCDA32D
:1042BC00EFF07F039080C4EFF0A374CDF0301022A8
:1042CC009062D0E09080C0F09062D1E09080C1F01C
:1042DC009062D2E09080C2F09062D3E09080C3F004
:1042EC00800C9080C074FFF0A3F0A3F0A3F090803A
:1042FC00017402F0906BC012259800000000906BC6
:10430C00BCE090804CF0906BBDE090804DF0906BD9
:10431C00BEE090804EF0906BBFE090804FF0A3E435
:10432C00F0A3F0A3F0A3F0908024F0A3F0A3F0A3EB
:01433C00F090
:01433D00225D
:1045FB008C258D26A907EAFDE975F018A424ACFFDC
:10460B00E5F034808F82F583EDF0EBFDE975F01862
:10461B00A4FFAEF024ACFBEE34808B82F583A3EDCC
:10462B00F08526828C83E0FDEF24A8FFEE3480FE1C
:10463B008F82F583EDF08526828C83A3E08F828EAB
:10464B0083A3F0852682852583A3A3E0FDE975F07E
:10465B0018A424A8FFE5F03480FE8F82F583A3A372
:10466B00EDF08526828C83A3A3A3E08F828E83A398
:04467B00A3A3F022E3
:064575008D2AAB07AA0627
:10457B00906BB8E0FCA3E0FDA3E0FEA3E0F52E8E6C
:10458B002D8D2C8C2BAE02AF038E838F8263A201F9
:10459B00E52D540744C0F583852E8263A201AF2A13
:1045AB00123437908000E020E5F9E4FCFDFEE52EA7
:1045BB00252AF52EEE352DF52DED352CF52CEC357C
:1045CB002BF52BC2A8908040E52BF0A3E52CF0A394
:1045DB00E52DF0A3E52EF0D2A89080007420F0AF6B
:0F45EB002EAE2DAD2CAC2B906BB812258CAF2AB9
:0145FA00229E
:064700008D25AB07AA069F
:10470600906BBCE0FCA3E0FDA3E0FEA3E0F5298EE0
:10471600288D278C26AE02AF038E838F8263A2017B
:10472600E528540744D0F58385298263A201AF2585
:10473600123437E4FCFDFEE5292525F529EE35285A
:10474600F528ED3527F527EC3526F526C2A8908005
:1047560058E526F0A3E527F0A3E528F0A3E529F020
:10476600D2A89080027420F0AF29AE28AD27AC26DF
:08477600906BBC12258CAF25ED
:01477E002218
:0241EE008F261A
:1041F000908001E030E5037F0022906BC0E0FCA3DB
:10420000E0FDA3E0FEA3E0F52A8E298D288C2790FF
:1042100065FC63A201E529540744C8F583852A8219
:1042200063A2017F0612344DE52A2406F52AE435FF
:1042300029F529E43528F528E43527F5279064FA8F
:1042400063A201E529540744C8F583852A8263A245
:1042500001AF2612344DE4FCFDFEE52A2526F52AA1
:10426000EE3529F529ED3528F528EC3527F527C257
:10427000A890804CE527F0A3E528F0A3E529F0A35A
:10428000E52AF0D2A89080017420F0AF2AAE29ADC3
:0B42900028AC27906BC012258CAF26D5
:01429B002200
:103E4700C2A89081E0E0F52505250525052505256E
:103E5700052505250525052505250525908010E05F
:103E6700F528A3E0F529A3E0F52AA3E0F52B908137
:103E7700E1E0F52505250525052505250525052564
:103E87000525052505250525908014E0F52CA3E0DB
:103E9700F52DA3E0F52EA3E0F52FD2A8E52EB52A40
:103EA70008E52FB52B037F0022E4F525E52E5407FF
:103EB70044E0F583852F8263A2019062F863A20133
:103EC7007F081234659062FA63A2019062AE63A222
:103ED700017F061233CE9062F8E0F526A3E0F527BE
:103EE700E4F5259062F8E0702AA3E024F8F525E5CB
:103EF7002E540744E0F583852F8274082582F582C6
:103F0700E43583F58363A2019062F863A201AF25CC
:103F1700123465AE26E4FCFDE52F2527F52FE52EA7
:103F27003EF52EED352DF52DEC352CF52CC2A89050
:103F37008014E52CF0A3E52DF0A3E52EF0A3E52FE3
:0B3F4700F0D2A89080007440F0AF257D
:013F5200224C
:10364900C2A89081E6E0F52505250525052505256E
:10365900052505250525052505250525908028E04D
:10366900F528A3E0F529A3E0F52AA3E0F52B90813D
:10367900E7E0F52505250525052505250525052564
:10368900052505250525052590802CE0F52CA3E0C9
:10369900F52DA3E0F52EA3E0F52FD2A8E4F525E555
:1036A9002EB52A0AE52FB52B05C2080237A7E52E44
:1036B900540744F0F583852F8263A2019062F86371
:1036C900A2017F081234659062F8E0F526A3E0F5BF
:1036D90027E527452670099080027410F07F0022A3
:1036E900906603E0FFF4602D9062FAE06F707690C7
:1036F9006604E0FF9062FBE06F706A906605E0FF88
:103709009062FCE06F705E906606E0FF9062FDE0FB
:103719006F602280509062FAE0906603F09062FB3D
:10372900E0906604F09062FCE0906605F09062FD1E
:10373900E0906606F09062F8E0702AA3E024F8F5BC
:1037490025E52E540744F0F583852F8274082582D8
:10375900F582E43583F58363A2019062F863A201DF
:10376900AF25123465AE26E4FCFDE52F2527F52F9C
:10377900E52E3EF52EED352DF52DEC352CF52CAF3E
:103789002BAE2AAD29AC28AB2FAA2EA92DA82CD354
:1037990012257B40099080027410F07F0022C2A894
:1037A90090802CE52CF0A3E52DF0A3E52EF0A3E500
:0C37B9002FF0D2A89080027440F0AF25E1
:0137C50022E1
:10393200C2A89081E3E0F525052505250525052585
:1039420005250525052505250525052590801CE06D
:10395200F528A3E0F529A3E0F52AA3E0F52B908151
:10396200E4E0F5250525052505250525052505257B
:103972000525052505250525908020E0F52CA3E0E9
:10398200F52DA3E0F52EA3E0F52FD2A8E4F525E569
:103992002EB52A0AE52FB52B05C209023A7AE52E81
:1039A200540744E8F583852F8263A2019060046383
:1039B200A2017F0E12347B906004E0F526A3E0F5AD
:1039C200279065FCE0FF90600CE06F706C9065FDE5
:1039D200E0FF90600DE06F70609065FEE0FF906028
:1039E2000EE06F70549065FFE0FF90600FE06F7023
:1039F20048906600E0FF906010E06F703C906601B6
:103A0200E0FF906011E06F7030906004E0702AA3D4
:103A1200E024F2F525E52E540744E8F583852F824C
:103A2200740E2582F582E43583F58363A2019060EA
:103A32000463A201AF2512347BAE26E4FCFDE52F20
:103A42002527F52FE52E3EF52EED352DF52DEC35FE
:103A52002CF52CAF2BAE2AAD29AC28AB2FAA2EA960
:103A62002DA82CD312257B5006E5274526700990F8
:103A720080017410F07F0022C2A8908020E52CF013
:103A8200A3E52DF0A3E52EF0A3E52FF0D2A89080B8
:063A9200017440F0AF25B5
:013A9800220B
:043F53008E338F34E6
:103F5700906BB8E0FCA3E0FDA3E0FEA3E0F53A8E8A
:103F6700398D388C37E53AFFE5395407FEE42FF5EC
:103F770036EE34C0F535853682F5837423F0053681
:103F8700E536700205355335C7F582853583740AE2
:103F9700F00536E536700205355335C79062C163C3
:103FA700A20185358385368263A2017F06123437E5
:103FB70074062536F536E43535F53585338385348E
:103FC7008263A20185358385368263A20112341B81
:103FD700908000E020E5F9E4FCFDFE906BB8E0F886
:103FE700A3E0F9A3E0FAA3E02FFFEE3AFEED39FDD7
:103FF700EC38FCEF2408FFE43EFEE43DFDE43CFC26
:10400700906BB812258CC2A8906BB8E0908040F0F6
:10401700906BB9E0908041F0906BBAE0908042F0ED
:10402700906BBBE0908043F0D2A89080007420F0A2
:014037002266
:064116008E338F348D355D
:10411C00906BB8E0FCA3E0FDA3E0FEA3E0F53B8EC2
:10412C003A8D398C38E53BFFE53A5407FEE42FF520
:10413C0037EE34C0F536853782F5837423F00537B6
:10414C00E537700205365336C7F582853683EBF0BA
:10415C000537E537700205365336C79062C163A246
:10416C000185368385378263A2017F06123437744A
:10417C00062537F537E43536F536853383853482B5
:10418C0063A20185368385378263A201AF35123471
:10419C0037908000E020E5F974082535F535FFE40B
:1041AC00FCFDFEE53B2FF53BEE353AF53AED3539A6
:1041BC00F539EC3538F538C2A8908040E538F0A3D5
:1041CC00E539F0A3E53AF0A3E53BF0D2A8908000E6
:1041DC007420F0AF3BAE3AAD39AC38906BB81225C9
:0141EC008C46
:0141ED0022AF
:064038008E2A8F2BAB0560
:10403E00906BB8E0FCA3E0FDA3E0FEA3E0F5318EAB
:10404E00308D2F8C2EE531FFE5305407FEE42FF531
:10405E002DEE34C0F52C852D82F5837423F0052DBD
:10406E00E52D7002052C532CC7F582852C83EBF0C1
:10407E00052DE52D7002052C9062C163A201852CE1
:10408E0083852D8263A2017F061234377406252D97
:10409E00F52DE4352CF52C532CC7E52A852D82857C
:1040AE002C83F0052DE52D7002052C532CC7F582BF
:1040BE00852C83E52BF0052DE52D7002052C532C58
:1040CE00C7908000E020E5F9E531240AF531E435AA
:1040DE0030F530E4352FF52FE4352EF52EC2A890AD
:1040EE008040E52EF0A3E52FF0A3E530F0A3E531F7
:1040FE00F0D2A89080007420F0AF31AE30AD2FAC6E
:07410E002E906BB812258C06
:014115002287
:104CF700E5D220E0FBC2AF438E2075D2028F8275CA
:0C4D07008300E0FFE4F5D2538EDFD2AF52
:014D1300227D
:104D4D00E5D220E0FBC2AF43D2028F82758300ED26
:0A4D5D00F075D25063D250D2AF229D
:10477F00E4FEEE04FF124CF774B92EF582E43462B6
:10478F00F583EFF00EBE3FEAE4FEEE247FFF124CFE
:10479F00F7742F2EF582E43461F583EFF0742F2E2A
:1047AF00F582E43461F583E0701B742F2EF582E4FB
:1047BF003461F5837420F074302EF582E43461F5A2
:1047CF0083E4F080040EBE80C1E49061AEF0FEAFD2
:1047DF0006124CF774AF2EF582E43461F583EFF0D7
:0447EF000EBEFEEB11
:0147F30022A3
:104D1400A2AF921FC2AF8C838D82EF12349343A251
:0C4D24002012349553A2DFA21F92AFFFB3
:014D30002260
:024CAF008F254F
:104CB100A2AF921FC2AFE4F5838D827406123493C2
:104CC100E52543A22012349553A2DFA21F92AF7FA4
:014CD10001E1
:014CD20022BF
:024CD3008F252B
:104CD500A2AF921FC2AFE4F5838D82740A1234939A
:104CE500E52543A22012349553A2DFA21F92AF7F80
:014CF50001BD
:014CF600229B
:1032F300A907E7FFA805EF93C3966008403B74FC5A
:103303002FFF80F00F08EF93C3966008402B74FBE8
:103313002FFF80E00F08EF93C3966008401B74FAF9
:103323002FFF80D00F08EF93D3966008400B74F9FA
:103333002FFF80C01F1F1F1F1FEF54FEF80303F74B
:10334300E893FC08E893FD08E893FE08E893FF225E
:1033530009E993C39D6008402974FB29F980F109A9
:10336300E993C39E6008401A74FA29F980E209E9D7
:1033730093D39F6008400B74F929F980D319191965
:103383001919E9C313C313FF22740093F8ECC3980C
:103393004024701F740193F8EDC39840197014749E
:0E33A3000293F8EEC398400E7009740393F87D
:1033B100EFC39840037F00227F0122EDF8E6F00879
:1033C100A3DFFA22EDF8E0F608A3DFFA22E0A36317
:1033D100A201F0A363A201DFF475A20022E0A363BE
:1033E100A201F0A363A201E0A363A201F0A363A27F
:1033F10001E463A201F0A363A201DFE175A200224F
:10340100E0A363A2016DFE936CFDEE058393FC15B1
:103411008363A201DFEA75A200227F00E493A36324
:10342100A201F00F600CA3E583C2E3F58363A2015F
:1034310080EA75A20022E0A363A201F0A3E583C2A2
:10344100E3F58363A201DFEE75A20022E0A363A28C
:1034510001F0A3E583C2E4D2E3F58363A201DFECCB
:1034610075A20022E583C2E3F583E0A363A201F024
:10347100A363A201DFEE75A20022E583C2E4D2E3D9
:10348100F583E0A363A201F0A363A201DFEC75A2BF
:103491000022F922C002C004C00612FFF0D006D0FB
:0434A10004D002222F
:104AD60020536572763A0020547261737353656E83
:104AE600644552520A00205265496E69742043415A
:104AF6004E0A002043414E283029203E20544F21A3
:104B06000A0020545520300A0020545520310A004E
:03001E00E4FF22DA
:104C2700C28DC2AF438901C28C906AAEE0FF7007A4
:104C3700F58A758CEE8016EFB40508E4F58A758C55
:104C4700B8800AEFB40A06E4F58A758C70D28CD264
:024C5700AF228A
:104B1600C28DC2AF438901C28C906AAEE0FF7014A9
:104B2600301E09F58A758CDCC21E801E758A667574
:104B36008CFC8016EFB40508E4F58A758CEE800AC5
:0F4B4600EFB40A06E4F58A758CDCD28CD2AF226C
:104D310012485B120022D21DE4F54E906BB6F0F5DD
:0C4D41003CF552124C27C21EE4F5502233
:104B8D00EF24FCF525200A127E4A7FD6123F537E74
:104B9D00627FFC7B01AD251241169062FC63A20180
:104BAD00906B3663A201AF251233CE85253CE4F51B
:034BBD004DC21BCB
:014BC00022D2
:0F4DA300D3EF6480948E5006E55270028F522237
:102CF500208D03022D91C28C201D03022DEAE53C97
:102D05006054743A254DF582E4346BF583E024056F
:102D1500F525D3940E4008E4F53CD21B022DEA7448
:102D250036254DF582E4346BF5837D3EAF251233B0
:102D3500C5E525254DF54DE53E30E702D21E124C81
:102D450027124984E54DC3953C5003022DEAE4F56D
:102D55003CD21B022DEAE54F6014906A9A7D3EFF36
:102D65001233C5124C27124984E4F54F8077E5529A
:102D750060149060047D3EFF1233C5124C27124942
:102D850084E4F552805F1248C0124C27123A998F9D
:102D950025EF6051124B16E4F550E551C3946E5082
:102DA5001874AF2551F582E4346AF583E52525517C
:102DB500F5517D3EAF251233BC300124E53E30E7A9
:102DC5000330101C9064FA7D3EAF251233BCAF254D
:102DD5001241EEEF700A200A077E4A7FDD123F534B
:102DE500AF25124C84300D1230000D0550E550D33F
:102DF50094F04004C2AF80FEC20D200203022F05ED
:102E050090660FE004F0700690660EE004F0E54E63
:102E15006031D394014004154E8028906BB6E004D0
:102E2500F0E0D39403400D200A077E4A7FEC123F61
:102E350053124D31200A077E4A7FF9123F53E4F5BC
:102E45004ED21D301C43E54F703F906A9A04F0A3A3
:102E55007408F0A37480F0A37401F0A37406F090D5
:102E65006B31E0906A9FF0906B32E0906AA0F09031
:102E75006B33E0906AA1F0906B34E0906AA2F0E4C5
:102E8500A3F0A3F0754F0BC21C301A72906B2FE0A4
:102E95007035E54F7031906A9A7442F0A37408F06A
:102EA500906B30E0906A9CF0906B35E0906A9DF0F5
:102EB500A37401F0754F06200A077E4B7F08123F69
:102EC50053906B2FE004F0906B2FE06402702FE5B8
:102ED5004F702B906A9A7402F0A37408F0906B30CF
:102EE500E0906A9CF0A3F0A37401F0754F06200AE8
:102EF500077E4B7F0F123F53906B2FE004F0C20209
:032F050012002691
:012F080022A6
:104BF400E551602CE49063F8F0A3E551F09065FB77
:104C0400E09063FAF0A37419F0906AAF63A2019084
:104C140063FC63A201AF511233CEE4F5517F01224C
:034C24007F0022EC
:0B4DB200301B05C21B7F01227F002286
:0100210022BC
:064DD500E4F551F53C225B
:100006007F01E4906107F0A3F0A3F0FEEF25E0FF87
:040016000EBE08F81A
:01001A0022C3
:104C59002043616E457247495400200A00204B5693
:104C690054210A002043616E457272434821000AAB
:0B4C7900000A20526571457272210094
:103A9900E59B541F6020200A1A7E4C7F59123F5320
:103AA900E59B541FFF7E007D031240387E4C7F63E7
:103AB900123F53E4F59BE5BA30E010E4F5B375B174
:103AC90080F5B2D21DF54E906BB6F0E5CFF47003D8
:103AD900023BD7752701E4F526E5CFF45527700396
:103AE900023BC5E526C454F0F5B1E5B2547F642024
:103AF9006003023B87E5B3540FF54285BC3E2010B5
:103B090016E5BD541FFF131313541FFFE5BD54E001
:103B190044184FF53F8006E5BD54E0F53FE5BDC4C7
:103B29003354E0FFE5BE131313541F4FF540E5BEB0
:103B3900C43354E0FFE5BF131313541F4FF54185F8
:103B4900A34385A34485A34585A34685A34785A3A8
:103B59004885A34985A34AE4F5B230100C85AE4BDC
:103B690085AF4C75B3D07F0F22E53E547EB53E0537
:103B790075B350800375B3D0E5422405FF22E5B241
:103B890030E60A200A077E4C7F66123F53E5B2549D
:103B99009F6023200A207E4C7F6D123F53AFB27E77
:103BA900007D03124038AFB37E007D031240387E9A
:103BB9004C7F78123F53E4F5B275B3D0E52725E081
:103BC900F5270526E526C394085003023AE27F004B
:013BD90022C9
:1049840020105875B180E4F5B3F5B2853EBCE5401E
:10499400C4135407FFE53F54E04FF5BDE5403333FE
:1049A4003354F8FFE541C41354074FF5BEE54133D2
:1049B400333354F8F5BF8543A38544A38545A385C4
:1049C40046A38547A38548A38549A3854AA3E54211
:0C49D400540F2450F5B3754E0AC21D228A
:1048C00020105F75B190E5B220E613200A107E4CEF
:1048D0007F7A123F53AFB27E007D03124038E4F579
:1048E000B3F5B274C8255AF582E43467F583E0F570
:1048F000BCE4F5BD74C9255AF582E43467F583E05C
:10490000FF33333354F8F5BE75BF78055A055A7432
:10491000C8255AF582E43467F583E07002F55A75CC
:03492000B350226F
:094DBD00EF6003C29622D2962297
:10485B0043AB01C2E8C2EAE4FFEFC454F0F5B1C3C5
:10486B00EF64809488500575B3D08003E4F5B3E40E
:10487B00F5B2F5BCF5BDF5BEF5BFF5C4F5C5F5C68E
:10488B00F5C7F5A3F5A3F5A3F5A3F5A3F5A3F5A339
:10489B00F5A30FBF0EC3906AAEE0FF25E0F5B4752C
:1048AB00B50C75B66C75A11275AB0275C13E75C3AF
:0448BB00FF75C203C0
:0148BF0022D6
:101F7800C7E0E3F0F3E7EEF7EDFBE920EEE1F0E090
:101F8800E73A20CACF20C8F1E5F2FC207620312EAE
:101F9800303328505050290A005452414E5A004DAF
:101FA800415842005254530044454C4159004D4F4A
:101FB8004445004B500054550043414E004E4F4D90
:101FC8004F44004154004454420043414E4D4F4E4B
:101FD8000054454C3A0049505300555345523A0075
:101FE8000D000A4F55542D5544503A000A4F555488
:101FF8002D5544503A4B5654000A4F55543A002038
:102008004348415021212000446973636F6E6E6517
:1020180063746564210A00536574205254530A009E
:102028004D6F64656D20696E6974266469616C0A18
:10203800004E4E45435400436F6E6E6563740A004C
:102048000ACFEEE2F2EEF020EFE5F0E5E4E0F7E8A3
:10205800000A484921000A5265714C43503237380A
:10206800000E0206000A000007020802000A50419A
:1020780050000A5265714C435033000A03060000B1
:102088000000000A435243204552523A20000A49B0
:102098004E3A000A20494E2D5544503A000A204530
:1020A80052524B56543A000A494E2D49503A004D67
:1020B8004F44454D204543484F210A200049434D90
:1020C800500A0050696E672D5265710A0050696E9A
:1020D800672D5265706C0A003F3F3F0A0049504324
:1020E800502D5245510A00495043502D41434B0051
:1020F800495043502D52454A00495043502D4143C1
:102108004B282049502052454144592120290A0092
:102118000A495043502D4E414B28495020414444D0
:1021280052293A000A495043502D5245510049500E
:1021380043502D52454A0A00495043502D544552A8
:102148004D0A004343502D5245510A004343502D38
:10215800524550004C43502D5245510A004C4350B3
:102168002D5245512D41434B004C43502D52455162
:102178002D4E414B00080304C023004C43502D5200
:1021880045512D52454A004C43502D41434B0A00BE
:102198004C43502D4E414B0A004C43502D54455250
:1021A8004D2D5245510A005041502D5265710A007B
:1021B800504150005041502D41434B0A005041506E
:1021C8002D4E414B0A000089129B24AD36BF48C1F1
:1021D8005AD36CE57EF78108931AA52CB73EC940FF
:1021E800DB52ED64FF76028B109926AF34BD4AC3EB
:1021F80058D16EE77CF5830A9118A72EB53CCB42DF
:10220800D950EF66FD74048D169F20A932BB4CC5CA
:102218005ED768E17AF3850C971EA128B33ACD44BE
:10222800DF56E960FB72068F149D22AB30B94EC7AA
:102238005CD56AE378F1870E951CA32AB138CF469E
:10224800DD54EB62F97008811A932CA53EB740C99A
:1022580052DB64ED76FF89009B12AD24BF36C1487E
:10226800D35AE56CF77E0A8318912EA73CB542CB6A
:1022780050D966EF74FD8B029910AF26BD34C34A5E
:10228800D158E76EF57C0C851E9728A13AB344CD4A
:1022980056DF60E972FB8D049F16A920BB32C54C3E
:1022A800D75EE168F37A0E871C952AA338B146CF2A
:1022B80054DD62EB70F98F069D14AB22B930C74E1E
:1022C800D55CE36AF17800112332465765748C9D1A
:1022D800AFBECADBE9F810013322564775649C8DFE
:1022E800BFAEDACBF9E82130021367764455ADBCAE
:1022F8008E9FEBFAC8D93120120377665445BDACDE
:102308009E8FFBEAD8C94253617004152736CEDF89
:10231800EDFC8899ABBA5243716014053726DECFBD
:10232800FDEC9889BBAA6372405125340617EFFE6D
:10233800CCDDA9B88A9B7362504135241607FFEE9D
:10234800DCCDB9A89A8B8495A7B6C2D3E1F0081959
:102358002B3A4E5F6D7C9485B7A6D2C3F1E018097D
:102368003B2A5E4F7D6CA5B48697E3F2C0D129382D
:102378000A1B6F7E4C5DB5A49687F3E2D0C139285D
:102388001A0B7F6E5C4DC6D7E5F48091A3B24A5B09
:1023980069780C1D2F3ED6C7F5E49081B3A25A4B3D
:1023A80079681C0D3F2EE7F6C4D5A1B082936B7AED
:1023B80048592D3C0E1FF7E6D4C5B1A092837B6A1D
:1023C80058493D2C1E0F2145000000000040007FA9
:1023D800110000FFFFFFFFFFFFFFFF03CC03CC004E
:1023E800000000007C2B2B2B7C0D6174680D7C6138
:1023F800747A0D7C61746400FF1FA1FF1FA7FF1F83
:10240800ACFF1FB0FF1FB6FF1FBBFF1FBEFF1FC1E2
:10241800FF1FC5FF1FCBFF1FCEFF1FD2FF1FD9FF16
:052428001FDEFF1FE2B2
:084DC6007E1F7F78123F53228B
:03002300022ACBE3
:0B2ACB00C0E0C083C082C0D075D018EE
:102AD600209803022BD4C298755601AF992014038F
:102AE600022BA020110FEF647E6003022BD4D211BB
:102AF600D291022BD4301508C215631F20022B8FEA
:102B0600BF7D05D215022BD4BF7E1CE50B547F700A
:102B160003022BD4906801E50BF0630B80530B8006
:102B2600C211C291022BD4E50B547FFED3940250FE
:102B360058EE7017EFF46013AE0B050B74302EF5DC
:102B460082E43468F58374FFF00513E50B547FFEC9
:102B5600BE0118EF64036013AE0B050B74302EF53F
:102B660082E43468F5837403F00513E50B547FFEA5
:102B7600BE0216EF30E012AE0B050B74302EF58256
:102B8600E43468F583E4F005137430250BF582E42C
:102B96003468F583EFF0050B80347430250BF5822D
:102BA600E43468F583E0B51F22906801E0701C05E7
:102BB6000B7430250BF582E43468F583E0700F90D2
:102BC60067F9F0906801E50BF08003750B0020991A
:102BD60003022CEC201203022CEA201403022CB36D
:102BE600300F63E512B4FF0D75997E051275160058
:102BF600D290022CEAE5166007F599751600802E2C
:102C060074072512F582E43468F583E0F516C3945B
:102C160020400BE516647D6005E516B47E087599BF
:102C26007D63162080068516997516000512E51235
:102C3600C3941D5003022CEAE5166003022CEAC277
:102C46000FF512022CEA9067C7E0FF65126005E5F2
:102C560012B4FF0CE516700875997E0512022CEA6F
:102C6600E512D39F400CE5167008C212D219C29025
:102C76008072E5166007F599751600806774302531
:102C860012F582E43469F583E0F516C39420400B0F
:102C9600E516647D6005E516B47E0875997D6316B4
:102CA6002080068516997516000512803774302522
:102CB60012F582E43469F583E0FF7008C212D21976
:102CC600C2908020D290EFB47C090512755332C2AF
:102CD600128011AF12051274302FF582E43469F5B3
:062CE60083E0F599C2999C
:092CEC00D0D0D082D083D0E032B8
:10135900C218C217C210906A30E4F0A37478F0E49E
:1013690090669FF078767C667D017BFF7A2379EC25
:10137900122783E49067FBF0A3F09067FEF0A3F0D7
:10138900C216906AAEF09067F8F0906BCC7467F073
:10139900A374C8F0906BCCE475F00112247385F046
:1013A90082F58374C4F0906BCCE475F00112247358
:1013B90085F082F583E4F0906BCC75F0011224730B
:1013C90085F082F58374C4F0906BCCE475F001125A
:1013D900247385F082F5837401F0906BCCE475F089
:1013E9000112247385F082F58374C8F0906BCCE404
:1013F90075F00112247385F082F583E4F0906BCCCB
:1014090075F00112247385F082F58374C8F0906B2E
:10141900CCE475F00112247385F082F5837401F030
:10142900906BCCE475F00112247385F082F5837416
:10143900C2F0906BCCE475F00112247385F082F54B
:1014490083E4F0906BCC75F00112247385F082F57A
:101459008374C2F0906BCCE475F00112247385F0AB
:1014690082F5837401F0906BCCE475F0011224735A
:1014790085F082F583E4F0906BCC75F0011224734A
:1014890085F082F583E4F0F55A906BC4F0906BC453
:10149900E075F003A42400F582E43424F583E49391
:1014A900FB740193FA740293F912242D7003021A42
:1014B9005FE4906BC6F0A3F0906BC5F0906BC5E04C
:1014C900242FF582E43461F583E0FF7003021A5694
:1014D900906BC4E075F003A42400F582E43424F58C
:1014E90083E493FB740193FA740293F9906BC6E059
:1014F900F582758300122446FEEFB5060F906BC77F
:101509007401F0906BC6E004F0021A4D906BC7E0CD
:101519007003021A4DEE6003021A44906BC4E0B4E2
:101529000F004003021A56901537F8282873021540
:10153900640215B1021A56021A56021A56021A56AE
:10154900021A560216C80216F902170202175702A2
:10155900175C0217610217D6021937906BC5E02490
:101569002FF9E43461FA7B01C0031B8B287529002C
:10157900752A00E4F52BD0031234A5906BC8122507
:101589008C906BC8E0F8A3E0F9A3E0FAA3E0FB7F35
:10159900007E8C7D0A7C001224C5122557906A981A
:1015A900EEF0A3EFF0021A56906BCC7467F0A374B7
:1015B900C8F0906BC5E0242FF582E43461F583E02F
:1015C90024D0F55AC394014007E55AD3940840033F
:1015D900E4F55AE55A6028906BCCE475F0011224C1
:1015E9007385F082F58374C4F0155A906BCCE47559
:1015F900F00112247385F082F583E55AF080D490C6
:101609006BC5E02430F582E43461F583E024D0F53C
:101619005AC394014007E55AD394084003E4F55AA4
:10162900E55A6028906BCCE475F00112247385F0BB
:1016390082F58374C8F0155A906BCCE475F00112E9
:10164900247385F082F583E55AF080D4906BC5E068
:101659002431F582E43461F583E024D0F55AC3944A
:10166900014007E55AD394084003E4F55AE55A6066
:1016790028906BCCE475F00112247385F082F58310
:1016890074C2F0155A906BCCE475F001122473857D
:10169900F082F583E55AF080D4906BCCE475F001C3
:1016A90012247385F082F583E4F0906BCC75F00118
:1016B90012247385F082F583E4F0F55A021A5690E4
:1016C9006BC5E0242FF9E43461FA7B01C0031B8B5D
:1016D90028752900752A00E4F52BD0031234A5904A
:1016E9006BC812258C906BCBE0906AAEF0021A564B
:1016F9009067F87401F0021A56906BC5E0242FF92F
:10170900E43461FA7B01C0031B8B28752900752A13
:1017190000E4F52BD0031234A5906BC812258CE494
:10172900FFFEFDFC906BC8E0F8A3E0F9A3E0FAA383
:10173900E0FBD312257B400F906BCAE0FFA3E0903A
:101749006A30CFF0A3EFF0D218C217021A56D21698
:10175900021A56D210021A56E4F55A906BC5E024C3
:101769002FF582E43461AF82906BCCF0A3EFF09057
:101779006BCCE0FEA3E0F5828E83E0FF6420601568
:10178900EF6012906BCDE004F07006906BCCE00432
:10179900F0055A80DA906BC5E0242FF9E4346175BD
:1017A9002801F529892A752B00855A2C7B017A662F
:1017B90079761244EC7528FF75291F752AE87B0193
:1017C9007A6679761249E0E4F55A021A56906BC5A1
:1017D900E0242FF582E43461AF82FE906BCCF0A354
:1017E900EFF0AA06F97B01C0031B8B287529007548
:1017F9002A00E4F52BD0031234A5906BC812258C6E
:10180900906BCBE09067FBF0906BCCE0FEA3E0F52A
:10181900828E83E0FF642E6015EF64206010906B68
:10182900CDE004F07006906BCCE004F080DA906BA8
:10183900CDE004F07006906BCCE004F0906BCCE046
:10184900FEA3E0AA06F97B01C0031B8B28752900BA
:10185900752A00E4F52BD0031234A5906BC8122524
:101869008C906BCBE09067FCF0906BCCE0FEA3E032
:10187900F5828E83E0FF642E6015EF64206010907E
:101889006BCDE004F07006906BCCE004F080DA9048
:101899006BCDE004F07006906BCCE004F0906BCC5B
:1018A900E0FEA3E0AA06F97B01C0031B8B2875297A
:1018B90000752A00E4F52BD0031234A5906BC812E9
:1018C900258C906BCBE09067FEF0906BCCE0FEA38B
:1018D900E0F5828E83E0FF642E6015EF64206010CE
:1018E900906BCDE004F07006906BCCE004F080DAE8
:1018F900906BCDE004F07006906BCCE004F0906B37
:10190900CCE0FEA3E0AA06F97B01C0031B8B287576
:101919002900752A00E4F52BD0031234A5906BC871
:1019290012258C906BCBE09067FFF0021A56E4F514
:101939005A906BC5E0242FF582E43461AF82906B35
:10194900CCF0A3EFF0E490669FF0906BCCE0FEA39F
:10195900E0F5828E83E0FF643A6017EF642060123D
:10196900906BCDE004F07006906BCCE004F0055A62
:1019790080D890669FE55AF0A3F0906BC5E0242FBC
:10198900F9E43461752801F529892A752B00855AEE
:101999002C7B017A6679A1124A3874A1255AF582FD
:1019A900E43466F583E4F0906BCDE004F0700690C2
:1019B9006BCCE004F0E4F55A906BCCE0FEA3E0F5C3
:1019C900828E83E0FF64206015EF6012906BCDE09A
:1019D90004F07006906BCCE004F0055A80DA7B01C4
:1019E9007A66799F124D7E74A02FF58274663EF552
:1019F90083E4F07B017A66799F124D7E749F2FF5FF
:101A09008274663EF583E55AF02406FF90669FE0EE
:101A19002FF0A3E0FF906BC5E02F2430F9E4346187
:101A2900752801F529892A752B00855A2C7B017A9D
:101A390066799F1244ECE4F55A8012E4906BC7F082
:101A4900906BC6F0906BC5E004F00214C5906BC4AE
:061A5900E004F002149607
:011A5F002264
:10446000E4F50A9067F9F0F50C906A31E024F9FE62
:10447000906A30E034FF906A96F0A3CEF090669E8A
:104480007437F090682F7405F0E4FF124DBDC2122E
:10449000C20FC219C20FC211C215C213E4F51290A5
:1044A00067C7F0F553F50BF556906A9874FFF0A3C3
:1044B00074F4F0121359C2ADE4F5C9D2CDD2CCC216
:1044C000C9C2CAF5CDF5CC906A98E0F5CBA3E0F56A
:1044D000CA85CBCD85CACCD29ED29CD2CAC2ACC230
:0C44E00098C29975B81075B710D2AC22C4
:0100220022BB
:104C840030160BE53EB44206E5416402601CE511B2
:104C9400C39450501574102511F582E43466F583DD
:0B4CA400EF2511F5117D3E1233BC22FC
:1037C6000515906814E02404FFE43401FE906816A1
:1037D600E07C002FFFEC3EFE906818E02FFFEC3EE9
:1037E600FE90681AE02FFFEC3E906803F0A3EFF01E
:1037F600AF17E5152517FFEC33CF242DCF3400FE88
:10380600906815E02FFFEC3EFE906817E02FFFEC66
:103816003EFE906819E02FFFEC3EFE90681BE02FFD
:10382600FFEC3E906805F0A3EFF0906803E0F52A00
:10383600A3E0F52BA3E0FEA3E0FDAC06E52A2DFDF3
:10384600E43CFC252BF52BE433F52AAB052BFDE4F4
:1038560033FC252BF52BE4352AF52AE52BF4906865
:1038660012F0AF05EFF4A3F0E517241C90680BF0F7
:10387600E5172408906821F090680DE515F074FFAF
:10388600F50DF50E75101D906A3263A20190693030
:1038960063A201AF171233CE90680763A20190218D
:1038A600CE63A201AF10AE0FAD0EAC0D1234018F78
:1038B600108E0F8D0E8C0D85171090693063A20146
:1038C6009021CE63A201AF10AE0FAD0EAC0D123437
:1038D600018F108E0F8D0E8C0DE50EF4FF743025C2
:1038E60017F582E43469F583EFF0E50DF4FF7431E2
:1038F6002517F582E43469F583EFF0E51724029085
:1039060067C7F0200A177E1F7FEA123F537E697F42
:10391600309067C7E024FEFDE4FB1241167512FFE6
:0B392600D20FD212C2992099FDD29955
:013931002273
:023BDA00A90739
:103BDC000515906814E02404FFE43401FE90681687
:103BEC00E07C002FFFEC3EFE906818E02FFFEC3ECF
:103BFC00FE90681AE02FF52BEC3EF52AE5152430E3
:103C0C00FFE433FE906815E02FFFEC3EFE90681742
:103C1C00E02FFFEC3EFE906819E02FFFEC3EFE908B
:103C2C00681BE02FFFEC3EAD07FCE52A2DFDE43CC4
:103C3C00FC252BF52BE433F52AAB052BFDE433FCEB
:103C4C00252BF52BE4352AF52AE52BF4906812F098
:103C5C00AF05EFF4A3F090680B741FF0906821741B
:103C6C000BF090680DE515F074FFF50DF50E751061
:103C7C001D906930E9F0B9820AA37401F0A3E51430
:103C8C00F08007E4906931F0A3F090680763A2011B
:103C9C009021CE63A201AF10AE0FAD0EAC0D12345D
:103CAC00018F108E0F8D0E8C0D7510039069306383
:103CBC00A2019021CE63A201AF10AE0FAD0EAC0DE0
:103CCC001234018F108E0F8D0E8C0DE50EF4906951
:103CDC0033F0E50DF4A3F09067C77405F0200A17D4
:103CEC007E1F7FF4123F537E697F309067C7E024BC
:103CFC00FEFDE4FB1241167512FFD20FD212C299CF
:053D0C002099FDD29991
:013D1100228F
:104D930074302512F582E43469F583EFF0051222AD
:082F09008E2A8F2B8D2C8B2DDD
:102F1100E4F5122013127FFF124D937F03124D939C
:102F2100E52AFF124D93800AE52AFF7E0060031215
:102F31004D93AF2BE52B124D93E52B6421452A6070
:102F4100030230667F45124D93E4FF124D93E41264
:102F51004D93AB2EAA2FA93012242D240CFF124D14
:102F6100937F88124D937F10124D937F40124D93A2
:102F7100E4FF124D937F7F124D93AF2D124D93AB12
:102F81002EAA2FA930900001122446FF7E009068DE
:102F910014E0248CFDE43401FC906816E07A002DE5
:102FA100FDEA3CCD2FFFEE3DFEAA2F900003122437
:102FB100467C002FF532EC3EF53112242D241CFF06
:102FC100E433FEEF252DFFEC3EFE906815E02FFF68
:102FD100EC3EFE906817E02FFFEC3EFE90000212DF
:102FE10024462FFFEC3EFE9000041224462FF52BC1
:102FF100EC3EF52AE531252BF52BE4352AF52A257A
:1030010032F532E433F531252BF52BE433F52A255E
:1030110032F532E43531F531E532F4FF124D93E505
:103021002BF4FF124D93906814E0FF124D939068BA
:1030310015E0FF124D93906816E0FF124D939068D2
:1030410017E0FF124D93AB2EAA2FA93012242D2485
:10305100FCF532E434FFF53174012530F530E43507
:103061002FF52F8021AF2C124D93AF2D124D93E4EC
:10307100FF124D93AB2EAA2FA93012242D24FDF55A
:1030810032E434FFF531E53245316022E532153263
:1030910070021531AB2EAA2FA93012242DFF124D2B
:1030A1009374012530F530E4352FF52F80D874FF66
:1030B100F50DF50E85121090693063A2019021CEB5
:1030C10063A201AF10AE0FAD0EAC0D1234018F1023
:1030D1008E0F8D0E8C0DE50EF4FF124D93E50DF460
:1030E100FF124D939067C7E512F0200A157E207FED
:1030F10001123F537E697F309067C7E0FDE4FB1208
:1031010041167512FFC20FD212C2992099FDD299B0
:01311100229B
:043D12008E2A8F2B3B
:103D1600752D08752E08752F019066CEE02404F5E2
:103D26002CE52DC3952C4003023DB274C7252DF515
:103D360082E43466F583E06403703374C9252DF597
:103D460082E43466F583E0B4C01074CA252DF5828A
:103D5600E43466F583E0642360149066C9E0B4C079
:103D66000D200A077E207F07123F537F022274C769
:103D7600252DF582E43466F583E014FF74017E0098
:103D8600A807088005C333CE33CED8F9FFE52A5EEF
:103D9600FEE52B5F4E7002F52F74C8252DF582E4E3
:103DA6003466F583E0252DF52D023D27E52F6003CA
:103DB600023E44752D08E52DC3952C507674C72513
:103DC6002DF582E43466F583E014FF74017E00A8C5
:103DD60007088005C333CE33CED8F9FFE52A5EFE49
:103DE600E52B5F4E703B74C8252DF582E43466F5ED
:103DF60083E0F52FE52DC3952C50BBE52F60B774F6
:103E0600C7252DF582E43466F583E0FF74C7252EB9
:103E1600F582E43466F583EFF0052E152F052D8027
:103E2600D374C8252DF582E43466F583E0252DF597
:103E36002D8083E52E24FC9066CEF0E4F52FAF2F7F
:013E46002259
:1000260030002DC20005099067F9E0600214F090D7
:100036006A30E0FEA3E0FFD3906A97E09F906A964D
:10004600E09E500CA3E004F07006906A96E004F07F
:10005600E553B4010CE4F553D212C2992099FDD2AE
:100066009930120DE509D394064009C212D21980BF
:1000760003E4F509906A30E0FEA3E0FFC3906A97B7
:10008600E09F906A96E09E5006E508941E404C203C
:100096000A077E207F10123F53C217E4FF124DBDA0
:1000A6009067F8E0600890669E7404F08005E4901E
:1000B600669EF0E4906A96F0A3F0C214F50B906881
:1000C60001F09068307455F09067F97402F0E4F529
:1000D6000AF508C21390660EF0A3F030170302016A
:1000E600AF9067F9E060030201AF90669EE014608E
:1000F6003324FE607A240360030201AFE4906A961B
:10010600F0A3F07F01124DBD90669EE004F090676B
:10011600F97401F0300A030201AF7E207F1F123FFF
:10012600530201AF200A077E207F28123F53783002
:100136007C697D017B017A66797612278378307C2B
:10014600687D017BFF7A207939122783E4F50B90CD
:100156006801F0F512D212C2992099FDD2999066E3
:100166009EE004F0E004F09067F9740AF0803A909B
:100176006801E0700A906A31E09067F9F0802A2001
:100186000A077E207F3F123F53E4F50B906801F08B
:1001960090669EE004F0E4906A96F0A3F0D217D23F
:1001A60014F51390660EF0A3F0301902C21930123E
:1001B600030203D3E55360030203D32017030203AC
:1001C600D3E50A64086003020286E50C6018B401F0
:1001D6000A050C7F82123BDA0203D3E4F50C7F8317
:1001E600123BDA0203D39067F9E0604CD390660FB6
:1001F600E094BC90660EE0940250030203D3050817
:10020600E508D394054014750A077402F0A374BC7C
:10021600F0E4906A96F0A3F00203D3E490660EF041
:10022600A3F0200A077E207F48123F539067F97497
:1002360064F01237C60203D3E51170030203D3E458
:10024600906A32F0A3E511F0906800E0906A34F00D
:10025600A37419F0E5112404F51790661063A20142
:10026600906A3663A201AF171233CE1237C6906773
:10027600F97464F0E4F51190660EF0A3F00203D36E
:10028600E50A64076003020322D390660FE094BC7C
:1002960090660EE0940250030203D3E4F0A3F090BC
:1002A6006A327480F0906A347401F0E4A3F0A30417
:1002B600F0A37430F0A3747BF0E4F526742F2526A2
:1002C600F582E43461F583E0FF643A601174392500
:1002D60026F582E4346AF583EFF0052680DE74396C
:1002E6002526F582E4346AF583747DF0743A252672
:1002F600F582E4346AF583E4F0E5262407906A3350
:10030600F0E5262409F5171237C60508300A030258
:1003160003D37E207F59123F530203D3E50A6004BC
:1003260064027035D390660FE094F490660EE09404
:100336000140260508E4F0A3F0200A077E207F5E30
:10034600123F53752EFF752F20753069AB087D015E
:100356007F217EC0122F098074E50A64047035D3AC
:1003660090660FE094F490660EE094014026E4F067
:10037600A3F00508200A077E207F75123F53752ECD
:1003860001752F6675309FAB087D017F237EC012F5
:100396002F098039E50A64067033D390660FE0941E
:1003A6006490660EE0940040240508E4F0A3F02073
:1003B6000A077E207F7A123F53752EFF752F207510
:1003C6003083AB087D017F217E80122F0930120316
:1003D600020BAA201703020BAA906801E0FF700324
:1003E600020BAAF527E4F0E5277003020BAA74FFB7
:1003F600F50DF50EE527547FC39513F510E5275443
:100406008025132430F582E43468F58363A20190D5
:1004160021CE63A201AF10AE0FAD0EAC0D123401AA
:100426008F108E0F8D0E8C0DE4F513E52754802466
:1004360030F582E43468AF82F5288F2953277FE5AB
:100446000E64B87004E50D64F06022300A03020BF6
:10045600AA7E207F8B123F53E4FBAD27AF29AE283F
:100466001241167D03AF0EAE0D12403822200A1837
:10047600E50A640860127E207F96123F53E4FBADC6
:1004860027AF29AE28124116E4906A96F0A3F090A1
:10049600669E7437F0852982852883A3A3E024808D
:1004A600700302077824C070030209EF24C06003BA
:1004B600020BAA852982852883A3A3A3E064216071
:1004C60003020BAAE529240DF582E43528F583E01D
:1004D6006411600302061274FFF50DF50E75100C1B
:1004E600E5292410FFE43528F5838F8263A2019065
:1004F60021CE63A201AF10AE0FAD0EAC0D123401CA
:100506008F108E0F8D0E8C0D906674E0650D700445
:10051600A3E0650E6003020612200A1A7E207F9B66
:10052600123F53E5292420FFE43528FEE52724DE83
:10053600FDE4FB124116E5292420F582E43528F571
:1005460083E054BFF526B48113E49067FDF090680C
:1005560000F0750A089067F9F0A3F022E526B48248
:1005660024E5292422F582E43528F583E0FF906806
:1005760000E0FEEF6E6003020BAAE004F0E4906771
:10058600F9F0F50822E5266003020BAAE50A6408DD
:100596006003020BAAE5292422F582E43528F583B7
:1005A600E0F5149067FDE065146026200A137E20AE
:1005B6007FA5123F539067FDE0FF7E007D0312404A
:1005C600389067FDE01465146003020BAA750C01F0
:1005D600229067FDE004F0750C01E5292421F582DF
:1005E600E43528F583E0F54FC3940F501BE5292425
:1005F60024FFE43528F5838F8263A201906A9A630B
:10060600A201AF4F1233CE22E4F54F22200A127E0A
:10061600207FAF123F53E4FBAD27AF29AE2812412E
:100626001685288385298263A2019066C763A20185
:10063600AF271233CEE50AC394074030906817E01F
:10064600FF9066DAE06F7032906816E0FF9066D928
:10065600E06F7026906815E0FF9066D8E0B5071A3F
:10066600906814E0FF9066D7E0B5070E300A0302E3
:100676000BAA7E207FB7123F53229066D4E0640116
:10068600600302076A200A077E207FC5123F53E5F2
:100696000AD394064003E4F5089066DFE064086038
:1006A60003020753200A077E207FCB123F53906632
:1006B600D7E09066DBF09066D8E09066DCF0906656
:1006C600D9E09066DDF09066DAE09066DEF090663E
:1006D600DA7410F0E49066DFF09066E5E0FF90666D
:1006E600E3E02FF50EE433F50DAF0EEF9066E1F083
:1006F600E50DA3F09066E4E0FF9066E2E02FFFE4EC
:1007060033FE9066E6E07C002FF50EEC3EF50DAF6D
:100716000EEF9066E2F0E50DFF9066E1E02FF50E34
:10072600E433F50DAF0EEFF0E50DFFA3E02FF090EB
:1007360066E1E0F4F0A3E0F4F0752E01752F66751E
:1007460030DA7B01E4FD7F21FE122F09229066DF5D
:10075600E06003020BAA300A03020BAA7E207FD5B3
:10076600123F5322300A03020BAA7E207FE0123F7B
:100776005322852982852883A3A3A3E064216003ED
:10078600020965E5292404F582E43528F583E02489
:10079600FE607814700302084014700302094914BD
:1007A600700302095724046003020BAA200A077E7D
:1007B600207FE5123F5385288385298263A2019015
:1007C60066C763A201AF271233CE7F047E00123DB7
:1007D60012EF6012200A077E207FEF123F53752624
:1007E60002750A06800D200A077E207FF8123F5305
:1007F600752604752E01752F667530CE9066CCE091
:10080600FBAD267F217E80122F0922200A077E213A
:100816007F01123F53E5292405F582E43528F58347
:10082600E065086003020BAA750A07F511F5089042
:10083600660E741FF0A37440F022200A077E217F03
:1008460018123F5385288385298263A2019066C7C3
:1008560063A201AF271233CE78077C687D017BFF48
:100866007A2379CE7E007F1D1226959066D1E09080
:100876006814F09066D2E0906815F09066D3E09028
:100886006816F09066D4E0906817F09067FBE090E9
:100896006818F09067FCE0906819F09067FEE090A9
:1008A600681AF09067FFE090681BF075100474FFFB
:1008B600F50DF50E90681863A2019021CE63A20192
:1008C600AF10AE0FAD0EAC0D1234018F108E0F8D22
:1008D6000E8C0D75100490681463A2019021CE63EE
:1008E600A201AF10AE0FAD0EAC0D1234018F108EFB
:1008F6000F8D0E8C0D75100490681C63A20190215B
:10090600CE63A201AF10AE0FAD0EAC0D1234018F47
:10091600108E0F8D0E8C0D906674E50DF0A3E50E0E
:10092600F0200A077E217F2C123F53752E01752F6A
:10093600667530CE9066CCE0FB7D017F217E80120D
:100946002F0922300A03020BAA7E217F36123F535B
:1009560022300A03020BAA7E217F40123F532285D2
:100966002982852883A3A3A3E064FD6003020BAA62
:10097600E5292404F582E43528F583E014600302B2
:100986000BAA200A127E207F96123F53E4FBAD2766
:10099600AF29AE28124116200A077E217F4B123F4F
:1009A6005385288385298263A2019066C763A201C5
:1009B600AF271233CE752604200A077E217F5412F4
:1009C6003F53E49066C7F09066CEE024069066C872
:1009D600F0752E01752F667530C89066CCE0FB7DEC
:1009E600087F217EC0122F0922852982852883A3AC
:1009F600A3A3E064216003020B3BE5292404F582EE
:100A0600E43528F583E024FE7003020ACE14700351
:100A1600020AF4147003020B03147003020B12246F
:100A2600046003020B31200A077E217F5C123F53CC
:100A360085288385298263A2019066C763A201AFD8
:100A4600271233CE530AFD7FC67E00123D128F2633
:100A5600EF604864026019200A077E217F65123F15
:100A660053752602E50AC39403503D430A028038B3
:100A7600200A077E217F71123F53E490660EF0A391
:100A8600F0752EFF752F2175307D9066CCE0FB7DCD
:100A9600037F217EC0122F09020B31200A077E2117
:100AA6007F83123F53752604E490660EF0A3F0751B
:100AB6002E01752F667530CE9066CCE0FBAD267F95
:100AC600217EC0122F098063E5292405F582E435CD
:100AD60028F583E065087053200A077E217F8F1270
:100AE6003F53E50AC394035042430A01803D530A2B
:100AF600FE200A377E217F98123F53802E200A0758
:100B06007E217F5C123F53530AFE801F200A077E18
:100B1600217FA1123F53E4906A96F0A3F0D217D238
:100B260014F51390660EF0A3F0F50AE50A64037057
:100B360073750A0422852982852883A3A3A3E0640A
:100B4600237061E5292404F582E43528F583E02441
:100B5600FE60391460442402704A200A077E217F11
:100B6600AF123F53E490660EF0A3F00508200A0783
:100B76007E217FB8123F53752E01752F6675309F03
:100B8600AB087D017F237EC0122F0922200A077E33
:100B9600217FBC123F53750A0522200A077E217F5A
:040BA600C5123F53E2
:010BAA002228
:1043E000020BABE493A3F8E493A34003F68001F23D
:1043F00008DFF48029E493A3F85407240CC8C333DE
:10440000C4540F4420C8834004F456800146F6DFAC
:10441000E4800B0102040810204080904DCEE47E21
:10442000019360BCA3FF543F30E509541FFEE493A1
:10443000A360010ECF54C025E060A840B8E493A368
:10444000FAE493A3F8E493A3C8C582C8CAC583CA93
:10445000F0A3C8C582C8CAC583CADFE9DEE780BE4B
:014DD40000DE
:10242D00BB010689828A83E0225002E722BBFE02AD
:09243D00E32289828A83E49322E0
:10244600BB010CE58229F582E5833AF583E022504B
:1024560006E92582F8E622BBFE06E92582F8E22295
:0D246600E58229F582E5833AF583E49322AF
:10247300A3F8E0C5F025F0F0E5821582700215831C
:06248300E0C838F0E82279
:1024890075F008758200EF2FFFEE33FECD33CDCC0A
:1024990033CCC58233C5829BED9AEC99E58298408D
:1024A9000CF582EE9BFEED9AFDEC99FC0FD5F0D66A
:1024B900E4CEFBE4CDFAE4CCF9A88222B800C1B994
:1024C9000059BA002DEC8BF084CFCECDFCE5F0CBD2
:1024D900F97818EF2FFFEE33FEED33FDEC33FCEB0B
:1024E90033FB10D703994004EB99FB0FD8E5E4F9C6
:1024F900FA227818EF2FFFEE33FEED33FDEC33FCB3
:10250900C933C910D7059BE99A4007EC9BFCE99AA6
:10251900F90FD8E0E4C9FAE4CCFB2275F010EF2FEB
:10252900FFEE33FEED33FDCC33CCC833C810D707EB
:102539009BEC9AE899400AED9BFDEC9AFCE899F826
:0E2549000FD5F0DAE4CDFBE4CCFAE4C8F922B9
:0E255700C3E49FFFE49EFEE49DFDE49CFC2295
:10256500EB9FF5F0EA9E42F0E99D42F0EC6480C8ED
:0625750064809845F0228D
:10257B00EB9FF5F0EA9E42F0E99D42F0E89C45F0B6
:01258B00222D
:0C258C00ECF0A3EDF0A3EEF0A3EFF022C2
:10259800A8828583F0D083D0821225AF1225AF128E
:1025A80025AF1225AFE473E493A3C583C5F0C583B3
:1025B800C8C582C8F0A3C583C5F0C583C8C582C88D
:0125C80022F0
:1049E0008B258A2689278B2B8A2C892DAB25052799
:1049F000E527AA267002052614F912242D70ED74FD
:104A0000FF2527F52774FF3526F526AB28052AE56F
:104A10002AAA297002052914F912242DFFAB2505B5
:104A200027E527AA267002052614F9EF1227A070A1
:084A3000DAAB2BAA2CA92D2200
:1044EC008B258A268927E4F52DF52ED3E52C94000F
:1044FC00E52B64809480406AAB25AA26A927852EDB
:10450C0082852D83122446600A052EE52E70E9055E
:10451C002D80E5AB28AA29A92A12242D6034052A5E
:10452C00E52A7002052914F912242DFFAB25AA26C1
:10453C00A927052EE52EAC2D7002052D14F5828CC5
:10454C0083EF1227B2E52C152C7002152B14452B7A
:10455C0070C1AB25AA26A927852E82852D83E4124E
:09456C0027B2AB25AA26A92722DB
:104A38008B258A268927E4F52DF52EE52C152CAE35
:104A48002B7002152B4E6033AB28AA29A92A1224F1
:104A58002DFFAB25AA26A927052EE52EAC2D700221
:104A6800052D14F5828C83EF1227B2EF60CD740107
:104A7800252AF52AE43529F52980C0AB25AA26A9D7
:024A88002722E3
:104D7E00E4FFFE12242D600C0FEF70010E09E97096
:054D8E00F20A80EF2293
:1034A5008B258A268927E4F531F530F52FF52EF59C
:1034B5002CF52DE529452A45286012EBC0E0EAC028
:1034C500E0E9C0E0AB28AA29A92A122823AB2505E3
:1034D50027E527AA267002052614F912242DF532B0
:1034E500C394094007E532D3940D40E1E5326420E9
:1034F50060DBE532B42D05432D038016E532B42B90
:1035050005432D01800C74FF2527F52774FF35260B
:10351500F526E52B60046410703FAB25AA26A92784
:1035250012242D64306009E52B702E752B0A802935
:10353500900001122446FF64786004EFB4581343E9
:103545002D01752B1074022527F527E43526F52660
:103555008007E52B7003752B08AB250527E527AA02
:10356500267002052614F912242DF532C394614004
:103575000AE532D3947A50035332DF74D02532F5FD
:1035850032C3940A400CE5329411406D74F925322A
:10359500F532E532D3952B5060432D0185313685C3
:1035A5003035852F34852E33AF2B7E00E4FCFDAB03
:1035B50031AA30A92FA82E1227D4C8ECC8C9EDC945
:1035C500CAEECACBEFCBE4FCFDFEEB2532F531EEBE
:1035D5003AF530ED39F52FEC38F52EAF31AE30AD8B
:1035E5002FFCAB36AA35A934A833D312257B50035B
:1035F50002355E432D0402355EE52D20E003E480AF
:103605002DE529452A4528601EAB25E52724FFF928
:10361500E52634FFFAEBC0E0EAC0E0E9C0E0AB28FC
:10362500AA29A92A122823E52D30E20774FFFFFEF7
:10363500FDFC22E52DAF31AE30AD2FAC2E30E103D0
:0436450002255722E1
:1025C900E709F608DFFA8046E709F208DFFA803EF4
:1025D90088828C83E709F0A3DFFA8032E309F608E1
:1025E900DFFA8076E309F208DFFA806E88828C834D
:1025F900E309F0A3DFFA806289828A83E0A3F608FF
:10260900DFFA805689828A83E0A3F208DFFA804ADA
:1026190080D280FA80C680D4806580F280318010B3
:1026290080A680EA809A80A880DA80E280CA803118
:1026390089828A8363A20188828C8363A201E493DD
:10264900A363A201F0A363A201DFF3DEF1800B898A
:10265900828A83E493A3F608DFF9ECFAA9F0EDFB8B
:102669002289828A8363A20188828C8363A201E022
:10267900A363A201F0A363A201DFF4DEF280DB8988
:10268900828A83E493A3F208DFF980CE88F0EF60B1
:10269900010E4E60C588F0ED2402B4040050BBF56C
:1026A90082EB2402B4040050B123234582239026EF
:0226B900197393
:1026BB00E709F60870FA8046E709F20870FA803EDF
:1026CB0088828C83E709F0A370FA807CE309F60813
:1026DB0070FA8074E309F20870FA806C88828C833C
:1026EB00E309F0A370FA806089828A83E0A3F6087D
:1026FB0070FA805489828A83E0A3F20870FA8048CA
:10270B0080D280FA80C680D4806180F2802F8010C6
:10271B0080A680EA809A80A880DA80E280CA802F27
:10272B0089828A8363A20188828C8363A201E493EA
:10273B00A363A201F0A363A20170F3800B89828AC9
:10274B0083E493A3F60870F9ECFAA9F0EDFB228968
:10275B00828A8363A20188828C8363A201E0A363D4
:10276B00A201F0A363A20170F480DD89828A83E465
:10277B0093A3F20870F980D088F0ED2402B4040022
:10278B0050C6F582EB2402B4040050BC23234582CF
:05279B002390270B73E1
:1027A000BB010689828A83F0225002F722BBFE0118
:0227B000F32212
:1027B200F8BB010DE58229F582E5833AF583E8F05D
:1027C200225006E92582C8F622BBFE05E92582C809
:0227D200F222F1
:1027D400E88FF0A4CC8BF0A42CFCE98EF0A42CFCA4
:1027E4008AF0EDA42CFCEA8EF0A4CDA8F08BF0A422
:1027F4002DCC3825F0FDE98FF0A42CCD35F0FCEB81
:102804008EF0A4FEA9F0EB8FF0A4CFC5F02ECD3945
:0F281400FEE43CFCEAA42DCE35F0FDE43CFC22B2
:10282300BB011A89828A83D0F0D0E0F8D0E0F9D0D6
:10283300E0FAD0E0FBE8C0E0C0F002287B5016E9E4
:10284300F8D083D082D0E0F9D0E0FAD0E0FBC082A8
:10285300C083022872BBFE16E9F8D083D082D0E091
:0F286300F9D0E0FAD0E0FBC082C08302288422C3
:09287200EBF608EAF608E9F6228B
:09287B00EBF0A3EAF0A3E9F0225E
:09288400EBF208EAF208E9F22285
:00000001FF
